:020000000528D1
:0800080081298B138316850189
:10001000860106148830810083129E0120308B00F7
:1000200003309B000C089C00013006058C001C0668
:10003000031D9D170B1D27280B118D0F27288E0AD6
:1000400006300E02031C27288D038E0386119D1F88
:1000500036289D131C1C6F2986110C3081000D0859
:1000600090000E088F008D018E01B1281B08031D22
:1000700012281F301D05031D5C28861912280E0842
:10008000031D462804300D02031C122817080E0217
:10009000031C122803194D28522818080D020318B2
:1000A000522812280130063C0E02031D5A28FF3048
:1000B0000D02031D861512281D1C6D288619662841
:1000C00021080D02031C12288615122822080D0291
:1000D000031C12281D10861112289D1C7E288619CB
:1000E000772823080D02031C1228861512282408DD
:1000F0000D02031C12289D10861112281D1D8F2829
:100100008619882825080D02031C12288615122836
:1001100026080D02031C12281D11861112289D1D90
:10012000A0288619992827080D02031C1228861575
:10013000122828080D02031C12289D11861112286E
:100140001D1E12288619AA2829080D02031C122830
:10015000861512282A080D02031C12281D1286116A
:1001600012281B08031D12280F0891001008920086
:100170009D011108031DC42818301202031C6529B3
:1001800080301202031C6A290310110C9300120C18
:1001900094000310930C940C0310930C940C11080E
:1001A000031DD628A0301202031CDF2814081202F7
:1001B00098001308031C130F11029700E428143051
:1001C00012029800110897001308990014089A0069
:1001D0001D141830A00010301A029F0018309F0222
:1001E000031C56299D141830A00718309F02031CC9
:1001F00043291D151830A00718309F02031C302911
:100200009D151830A00718309F02031C1D291D16CC
:100210001830A00710309F0718309F0203181329C9
:100220001A08AA0015292008AA0014302002A900E3
:100230001830A0021030183C9F079F1F262910304D
:100240009F07031826291A08A80028292008A800B3
:1002500014302002A7001830A0021030183C9F076D
:100260009F1F392910309F07031839291A08A60043
:100270003B292008A60014302002A5001830A00257
:100280001030183C9F079F1F4C2910309F07031800
:100290004C291A08A4004E292008A400143020027A
:1002A000A3001830A0021030183C9F079F1F5F2941
:1002B00010309F0703185F291A08A200612920083F
:1002C000A20014302002A100122897011430183C1B
:1002D0009800122897011430120298001228013059
:1002E000063C0E02031D7B29FF300D02031D7B29F6
:1002F00003309B0012281B080319802986159B03D5
:0403000012280900B6
:02400E00F13F80
:00000001FF
